:10000000F01F0010693700006537000065370000F9
:10001000653700006537000065370000000000000C
:100020000000000000000000000000006537000034
:10003000653700000000000065370000251500004E
:100040001113000011130000111300001113000020
:100050001113000011130000111300001113000010
:100060001113000011130000111300001113000000
:100070001113000061370000613700006137000094
:10008000DD150000F51500000D1600002516000016
:1000900061370000ED160000613700006137000095
:1000A00061370000613700006137000061370000F0
:1000B00061370000613700006137000061370000E0
:1000C00008B500230B60036000F0AEFD08BD08B565
:1000D0000A20002101F022FA08BD000038B5094BC2
:1000E0000D1C041C1968012001F0C8FA012001F060
:1000F000A5FA291C201C02F097FE012001F0AEFA9F
:1001000038BDC046A804001008B5074B0120196887
:1001100001F0B4FA012001F091FA02F01DFE012075
:1001200001F09CFA08BDC046A804001013B5962043
:10013000000201F019FB18480D210C2200F07EFC92
:1001400000F0BCFB15480021032200F0EDFC00F09C
:10015000BFFBFFF7D9FF1248124901F0E9FC002468
:1001600001F0A8FB002802D000F0FAFF00240A20CA
:1001700001F004FA684601A9FFF7A2FF009B002BDB
:1001800003D1094B01349C42EADDFFF7BDFF07486C
:1001900001F0CEFC13BDC046A73B0000983900001B
:1001A000A7390000B23900006F170000B93900000C
:1001B00073B5124B041C1249186803F057FB114920
:1001C0000090114A114B201C01F0BDFC00F00EFE06
:1001D000002812D000F02AFEFA218900051C03F045
:1001E00045FB061C201C01F0FBFC094B2018734347
:1001F0000849EB18321C01F0A6FC73BDAC040010DA
:1002000040420F00C4390000B2390000D13900006B
:1002100018FCFFFFD439000070B50D1C161C041C1F
:1002200000F04CFB0B480D210C2200F007FC281CB1
:10023000A1B2002200F078FC07480321062200F05A
:10024000FDFB301C0121092200F06EFC00F040FB98
:1002500070BDC046A73B0000623A000010B588B0F0
:10026000041C6846FFF7A4FF69466A46201CFFF796
:10027000D3FF08B010BD000073B518200021FFF7B0
:100280002DFF454E0024454D983600E0434D01209A
:1002900001F0E4F9002C01D0002000E0062001214B
:1002A00001F03CF9684601A9FFF70AFF009B002B0B
:1002B00021D1002CF0D13368002B0DD0384B0094A5
:1002C0001A6811321A6004E002F0F0FC009B01335E
:1002D0000093009B102BF7DD324BED18DED5182074
:1002E0000021FFF7FBFE2C4B94331C6863425C41FA
:1002F00000F0B8FACEE7002C03D0182BC7D100F0DD
:10030000EFFA009B182B30D1019BC22B08D1264B52
:100310000022196801311960022900D11A60019286
:10032000019B832B08D10020FFF798FFFFF7ECFE1D
:10033000FFF7CDFE00230193019B732B03D1FFF741
:10034000F5FE00230193019B322B0ED1174B0124A4
:100350001868201A00F07CFD201CFFF77FFFFFF7D4
:10036000D3FEFFF7B4FE00230193114B012019685F
:1003700001F084F9012001F061F90098019902F07F
:1003800053FD054B002494331B68002B00D07DE700
:1003900000F068FA012479E7B004001020BF0200E1
:1003A000DC0200100CFEFFFF8C01001004000010A6
:1003B000A804001013B501F043FC00F001FC00F0AC
:1003C0008FFA00F0D9FE3C24201CFFF747FF013CC8
:1003D0001E2001F0D3F8022CF6D102F089FB1E2377
:1003E00000930A2301931348134B1449002202F08F
:1003F00039FC00200421012200F0DAFE0020021C5A
:10040000042100F023FF00200521012200F0D0FE8E
:100410000020021C052100F019FF0948002100F00E
:1004200039FF0021074800F035FF00F06FFCFFF7AF
:1004300023FFC0461D370000DC020010C100000091
:10044000984004409C40044000B500E0013003782F
:10045000202BFBD000BD00B5031C303BDAB2092ACB
:1004600001D8181C08E020231843031C613B5738AF
:10047000052B01D90120404200BD70B50E1CFFF7CD
:10048000E3FF0025041C06E0FFF7E5FF002805DB7D
:100490002D010543013420780028F5D13560201C5A
:1004A00070BD000008B500F0C1FC011C014801F05E
:1004B0003FFB08BDDF39000070B5054E051C0E245A
:1004C000013C295D301C01F033FB002CF8D170BDDC
:1004D000EB39000000B5C300181A064BC0180723FB
:1004E000013BC25C002A03D1002BF9D1012000E0BE
:1004F000002000BD4C0500107FB52D4801F018FB11
:1005000000250326354219D1281CFFF7E3FF0028F8
:1005100010D0681CFFF7DEFF00280BD0A81CFFF7E7
:10052000D9FF002806D0E81CFFF7D4FF002801D02F
:1005300004350FE01F48291C01F0FAFA291C68460F
:1005400001F0E8FB6846FFF7B7FF1B4801F0F0FA3F
:100550006C1C251CFF2DD5DD184801F0E9FA184C5C
:10056000201CFFF7A9FF174D4221281C01F0E0FADB
:10057000201C0E30FFF7A0FF4321281C01F0D8FA01
:10058000201C1C30FFF798FF0F4801F0D1FA201C07
:100590002A30FFF791FF281C4E2101F0C9FA201CD8
:1005A0003830FFF789FF616D084801F0C1FA7FBD5F
:1005B000B2390000EE3900005B550000F739000049
:1005C000B0040010FD390000043A00000A3A0000AF
:1005D00070B50E1CFFF738FF0D25041C2078FFF7BF
:1005E0003AFF002807DB01347055013DF6D2201C8C
:1005F000FFF72AFF00E0002070BD000030B5464C38
:1006000087B023680868002B06D1444801F090FAAF
:1006100002F06EFA012357E0012B12D18379202BCF
:1006200007D0002B05D03E49062201F0ECFA002845
:1006300003D1394B1A6801326AE03A4801F078FA7E
:100640005EE00378412B1BD1374C0230211CFFF7B1
:10065000BFFF002854D00378422B51D1211C023017
:100660000E31FFF7B5FF00284AD00378432B47D15E
:10067000211C02301C31FFF7ABFF002849D13FE0BD
:100680004D2B23D1294D0230291CFFF7A1FF002853
:1006900036D003784E2B33D1291C02300E31FFF7B0
:1006A00097FF00282CD00378472B29D1023005A9C9
:1006B000FFF7E3FE059B002B22DB2A3D6B651C4800
:1006C0001C4901F035FA0023236022E005A9FFF759
:1006D000D4FE0378041C202B01D0002B10D1002560
:1006E000201C01A9FFF774FF0599041C691801A8D3
:1006F00001F024FB002C03D00135042DF0D108E0DB
:1007000002F0F6F90A480C4901F012FA024B0022F5
:100710001A6007B030BDC046B4020010163A00009F
:10072000B23900002C3A0000B0040010DA040010C6
:10073000383A0000423A0000453A000037B54C68AC
:1007400024E0201CFFF780FE01A9FFF796FE019B25
:10075000041C002B1DD0D8B2FF2B09DD00F000FADD
:10076000051C01980012C0B200F0FAF9019003E0F4
:1007700000F0F6F9002501900198002802D0291C0C
:10078000FFF7ACFC23785A1E9341E4182378002B22
:10079000D7D137BD08B5064A012113784B401370F5
:1007A00001D0044900E00449044801F0C1F908BD42
:1007B000950300104C3A00004F3A0000533A0000F5
:1007C00070B5051C01200821021C00F03FFD072424
:1007D000012601200821002200F038FD2A1C2241B8
:1007E00032400020022100F031FD01200821021CCE
:1007F00000F02CFD013CECD270BD10B50021041CB2
:100800000A1C022000F022FD201CFFF7D9FF10BDBA
:10081000F7B5012300930023019372B66C46061CC2
:1008200002AF01CC50235B421843C0B2FFF7E5FF93
:100830000020FFF7E2FF1020FFF7DFFFE020FFF7C7
:10084000DCFF002502200021012200F0FFFC705D8A
:100850000135FFF7B5FF842DF4D18436BC42E0D1D9
:1008600062B6F7BD08B5AC20FFF7C7FFAE20FFF7B3
:10087000C4FFA520FFF7C1FF08BD08B5AF20FFF7F3
:10088000BCFFA420FFF7B9FF08BD08B5AE20FFF7F5
:10089000B4FF08BD10B5041CF820FFF7AEFF201C04
:1008A000FFF7ABFF10BD10B5041C8120FFF7A5FFBB
:1008B0003F202040FFF7A1FF10BD000008B58422B3
:1008C00002480021520001F06BF908BD9D030010A1
:1008D00008B50248FFF79CFF08BDC0469D03001005
:1008E00008B50120021C082100F062FC0120021C56
:1008F000082100F0ABFC00200221012200F058FC8E
:1009000000200221012200F0A1FC0220002101228E
:1009100000F04EFC02200021012200F097FC022092
:100920000621012200F044FC02200621012200F0F1
:100930008DFC0320011C012200F03AFC0320011C65
:10094000012200F083FC0320011C002200F07EFC49
:1009500002200621002200F079FC0621012202205B
:1009600000F074FCFFF7AAFFFFF7B2FFA220FFF729
:1009700044FFA020FFF741FFC020FFF73EFF00200B
:10098000FFF788FF0A2000F0F9FD4020FFF735FF50
:100990002C20FFF732FF322000F0F0FD2E20FFF771
:1009A0002CFF322000F0EAFD2F20FFF726FF0A205F
:1009B00000F0E4FD2520FFF720FFAF20FFF71DFF2B
:1009C000A420FFF71AFF0020FFF76DFF08BD00000D
:1009D00000B50F290ED883280CD8CB0884225343A6
:1009E0000722C0181140044B80220A41111C1A5CD6
:1009F0001143195400BDC0469D030010F0B55B18AB
:100A0000DBB216E08425CC086C4307270F40802515
:100A100004193D41EFB2A6189C4605E0064BE518C7
:100A20002B7801343B432B70B442F7DB0131634632
:100A3000C9B29942E6D3F0BD9D03001000B5084B42
:100A40001860084B1970084B20211A70074B197059
:100A5000074BD1081970500701D00131197000BD42
:100A600098030010A5040010A7040010A6040010AD
:100A70009C030010F0B589B0059106925A2800D960
:100A80002020264B00241B78221CC01A244B1B68F4
:100A900004E002310C190132A4B2D2B2195D8242D3
:100AA000F7DB1B195B780391029300222CE000997D
:100AB0004B4303999A198A4214DA194A002512689D
:100AC00092191219D3189B7804930123049AAB400E
:100AD000134204D07919C9B20798FFF779FF01359D
:100AE000082DF2D101360837F6B2FFB206E00099C0
:100AF000059A069F8B18DBB20026079309490B78ED
:100B00009E42D4D3019A013201926B461B7902991D
:100B100000938B42EBD309B0081CF0BDA604001073
:100B2000980300109C030010F7B5061C0C1C0192E2
:100B300001F056F880B200900025832709E06B464B
:100B4000705DE1B21A79FFF795FF01302418A4B265
:100B50000135009AABB2934201D2A742EFD2F7BD62
:100B600000B50F23020918408000031F00D5283369
:100B7000002B0EDB511E032088428041404200289A
:100B800007D1242B06DC04218A1A0349CB18985C70
:100B900000E0002000BDC046AA3F000070B5064E30
:100BA000051C0024A05D054B291CC018013400F071
:100BB00071FB0A2CF6D170BDE63F000000400440F6
:100BC000F8B51020FFF7EAFF094C271C14372578E9
:100BD0006678281C311C002200F0EAFA0234281C36
:100BE000311C012200F032FBBC42F0D1F8BDC046FE
:100BF000D23F0000F8B50B4C271C143725786678D7
:100C0000281C311C012200F0D3FA0234281C311CAC
:100C1000002200F01BFBBC42F0D10020FFF7BEFF1A
:100C2000F8BDC046D23F0000F0B589B00024049062
:100C30000591FFF7C5FF02200721012206940794C2
:100C400000F0B6FA02200721221C00F0FFFA201C57
:100C50000B2100F0D1FAA04202D1182306930124FF
:100C60000021264D03916A782F78111C0192381CBF
:100C7000012200F09DFA381C0199002200F0E6FAEA
:100C800003231F4E029314E03078717800F0B4FA19
:100C9000002807D103991B4AA3008A5C18336946D0
:100CA0005A500134029A039B013A01330292039392
:100CB000023EE30F00210122A2424B41DBB28B42F4
:100CC00002D0029B8B42DFDA381C0199002200F02F
:100CD0006FFA0199381C012200F0B8FA0A4902356E
:100CE0008D42C0D1201E06D0069B049A0599136040
:100CF000079B01200B6009B0F0BDC046D23F000049
:100D0000A83F0000AA3F0000E63F000008B5012010
:100D1000021C0B2100F04CFA01200B21002200F0F4
:100D200095FA03200221012200F042FA0320022159
:100D3000002200F08BFA08BD37B5234B10211A684A
:100D4000051C8A431A60214B8022196892010A43CC
:100D50001A6001200B21002200F02AFA01200B2149
:100D6000002200F073FA1A4B9F211A68194C8A432B
:100D70001A601A6818491A60184B186802F076FD54
:100D80008023000218432A1C20600221032000F067
:100D90005DFA142000F0F2FB2368FF2293432360E6
:100DA00023680F4A134323600E4B1A680192019A7D
:100DB000002AFADA22680C4B13402360FFF7A6FFE3
:100DC00001980004800D3EBD3882044080800440BC
:100DD0009840044000C0014000093D00AC040010F0
:100DE000800000012CC00140FFFFFFF838B50E4C19
:100DF0002068002817DA00252560281CFFF79CFFD3
:100E0000281CFFF799FFA8420AD10120FFF794FFA1
:100E10000138C023FF385B00984201D801232360CA
:100E2000FFF774FF206838BD0000001008B5FFF719
:100E3000DDFF011E08D00120FFF77EFF011E03D059
:100E4000024802F013FD011C081C08BD50BB120033
:100E500010B500280DD0254B80211A688A431A60EE
:100E6000234A012311681942FCD0224B03221A6045
:100E700001E0204B1860204B012200211A6019600C
:100E80001A6019681142FCD01C4B01221A601C4ADE
:100E9000802114684902214311601A1C002804D1E2
:100EA000124B8024196821431960164B1968884237
:100EB0001AD01860002801D0134800E013481168C8
:100EC00002F086FC124C2121206002F0CFFC114B75
:100ED00018609620000200F047FCFA212068890083
:100EE00002F0C4FC00F030FB10BDC0463882044064
:100EF0000C8004407080044074800440788004407A
:100F00008080044004000010006CDC02001BB7006D
:100F1000AC040010A804001008B500F03BF9134B16
:100F200000211A68120B12031A60114B1A68120B77
:100F300012031A600F4B1A68120B12031A600E4B41
:100F40001A68120B12031A600C4B012219600C4B29
:100F50001A6019601A6019681142FCD0094B2322EB
:100F60001A600120FFF774FF08BDC04600800050E2
:100F700000800150008002500080035040800440F7
:100F8000448004400880044070B50F490F4800F0C9
:100F9000CFFD0F4800F0CCFD0E4E0F4D00242B1955
:100FA0006159DA68301C0A4B143400F0C1FD782C0A
:100FB000F5D10A4800F0BCFD00F0FCFA011C08481D
:100FC00000F0B6FD70BDC046B2390000F03F000031
:100FD0004140000001400000080000100C400000EB
:100FE0002E400000F0B53C4B8BB01D68002D3AD070
:100FF0003A4B02901B6801209B685DE00134237826
:10100000202BFBD0002B3AD0B30008336A469C500B
:101010000136FF2D01D135E001342378202B01D09A
:10102000002BF9D1202B02D1002323700134012E93
:101030001BD12A4F2A4B07223B6001923D1C09E03D
:101040002B680298196800F0EDFD002808D02B6885
:1010500014332B60019B013B0193002BF0D132E054
:101060003B681D7901E0041C2E1C2378002B06D060
:1010700000230722B2425B41DBB2002BBFD1002E1E
:101080001CD000E00025154C022E05D1039815490F
:1010900000F0C8FD002801D0AE420AD823681248EB
:1010A000D96800F045FD23681048196900F040FD3B
:1010B00004E02368F0B29B6802A99847064B1B68BE
:1010C000002B07D103E00198011CFFF75DFF0848E2
:1010D00000F02EFD0BB0F0BDB4020010BC020010F9
:1010E000080000103B4000003D4000003D3A000079
:1010F0004440000038B5041C154D0A2808D002D819
:1011000008281CD110E00D2802D07F2817D10BE051
:101110002B6800221A700F4800F00AFD0E4C201CAC
:10112000FFF760FF2C6012E02A680B4B9A420ED941
:101130000A48211C00F0FCFC2B68013B06E0074834
:10114000211C00F0F5FC2B681C7001332B6038BDAE
:10115000B802001041400000B401001050400000EF
:1011600008B503E000F084FBFFF7C4FF00F0A2FB2A
:101170000028F7D108BD000008B5034A034B044816
:101180001A6000F0D5FC08BDB4010010B8020010D0
:1011900044400000044B40211A680A431A60034B84
:1011A00001221A707047C04680800440C0020010BF
:1011B00070B50E4B061C1B780D1C141C002B01D1A6
:1011C000FFF7E8FF013E022E03D8094BB600F358A3
:1011D00000E0084B1A68012C03D1AC4014431C609A
:1011E00003E00124AC40A2431A6070BDC0020010AD
:1011F000D44000000080005038B50F4B051C1B7810
:101200000C1C002B01D1FFF7C5FF0020032D11D8C6
:10121000281C012302F0C8FA02040608074A04E069
:10122000074A02E0074A00E0074A1068A340184056
:10123000431E984138BDC046C0020010FC3F00501C
:10124000FC3F0150FC3F0250FC3F035070B50E4B79
:10125000061C1B780D1C141C002B01D1FFF79AFFF4
:10126000013E022E03D8094BB600F35800E0084BAC
:101270001A68012C03D1AC4014431C6003E0012424
:10128000AC40A2431A6070BDC0020010E0400000F4
:10129000FC3F005038B5084B041C1B780D1C002B7C
:1012A00001D1FFF777FF2368182293432360236857
:1012B0001D43256038BDC046C00200101F234209EF
:1012C000184001238340181C014B9200D0507047F6
:1012D00000E100E0054B3F221A60054B01221A6035
:1012E000044B40211A688A431A60704724800440E6
:1012F000D88004403882044008B5044B40211A6865
:101300008A431A60FFF7E6FF08BDC04638820440F2
:1013100008B50C4B1868FFF79BFD0B4B012252429E
:101320001A600A4A1268002A00D01A60084B1A682C
:1013300001321A60074A00231360074A1360C0464F
:1013400008BDC04604000010088204400C8204401E
:10135000C402001004C000403CC0004008B5FFF7C4
:1013600049FC0A480021FFF795FF09480021FFF7D3
:1013700091FF08480021FFF78DFF07480021FFF784
:1013800089FF06480021FFF785FF08BD084004409B
:1013900000400440AC400440144004401C40044061
:1013A000F7B50190FFF7DAFF474B01991A68474BF1
:1013B0001A60002901D0464B00E0464B464A042102
:1013C0001360464B464E1A68464F0A431A60019A0C
:1013D000002A54D0444B0025444C1D60444B201C33
:1013E0001D60291CFFF756FF281C09212A1CFFF746
:1013F000DFFE281C09212A1CFFF728FF3D4B802215
:101400001968032011431960236807218B43236067
:10141000236802210B43019923604B005B1899015B
:101420005B1801999B005B1833490B60334B1968BB
:1014300001431960324B334918680140196019683B
:1014400009200A431A60FFF739FF326880239B00A6
:101450001A43326001212C4A494211603A682249FC
:1014600013433B60294B02221A60294B01221A6068
:101470001D601A6018681042FCD001230B60254BD8
:1014800001221A600720FFF719FF0820FFF716FF57
:101490000A20FFF713FF0C20FFF710FF0B20FFF7C8
:1014A0000DFF32681C4B13403360019B002B03D1AE
:1014B0000122154B52421A603A68EC235B01134338
:1014C0003B6030BFF7BDC0463882044034820440E0
:1014D000BF180000FF1800003082044010ED00E04B
:1014E000008204400482044004C000406440044080
:1014F000044001408080044018C0004014C00040F7
:101500003CC000400FF0FFFF0882044070800440A0
:1015100074800440788004407FE2FFFF08B5FFF745
:101520003FFF08BD00B5064B1A6801321A601B6800
:10153000013303D1034B1A6801321A6000BDC04663
:10154000CC020010C802001000B5074B98420AD820
:10155000064A00231360064A01381060054A1360EA
:10156000054B07221A6000BDFFFFFF00CC020010F0
:1015700014E000E018E000E010E000E000B50C4AE4
:101580001368002800D10120C1438B4204D809E030
:1015900011688142FCD301E0591C08181168994276
:1015A000F6D203E01168C91A8142FBD300BDC046E0
:1015B000CC02001010B5064BFA211868054B8900C3
:1015C0001C6802F005F9044B5C43201810BDC046AE
:1015D000CC020010C802001037894100034B0122E1
:1015E0001A60034B1A6801321A60704700C000404D
:1015F000D0020010034B01221A60034B1A6801321B
:101600001A60704700000140D4020010034B012211
:101610001A60034B1A6801321A607047004001409B
:10162000D8020010034B01221A60034B1A680132E2
:101630001A60704700800140DC02001000B50028ED
:1016400003D1044B01221A6003E0012801D1024BAF
:10165000186000BD044001400480014000B500282E
:1016600002D1044B186004E0012802D1024B002291
:101670001A6000BD044001400480014010B50028FC
:101680000FD1124B80221C68920022431A60104B2B
:10169000032218600F4B19600F4B1A608022D20290
:1016A00011E0012811D1094B80221868D2000243B1
:1016B0001A600A4B00221A60094B03221960094B79
:1016C0001A6080221203084B1A6010BD808004400B
:1016D000D80200101840014014400140DC02001004
:1016E000188001401480014000E100E008B5184B6B
:1016F0001A680E231340062B0DD1164B9E221B6831
:10170000DBB2134204D0144A5360144B1B681EE032
:10171000D9071CD501E0042B05D1104B1868C0B2C5
:1017200000F0B7F813E00C2B06D10B4B8022596860
:1017300052000A435A600AE0022B08D1054B1A688E
:10174000054B910601D5002200E001229A6008BDF8
:101750000880004014800040E0020010008000403B
:1017600000487047E002001070B52A4C2A4B8022D6
:101770009203DA6700219022061C201C00F010FA68
:101780000023A36000F06EF8244B07251A68244C50
:10179000AA431A601968012211431960214B196884
:1017A000A94319601968114319601F4B80211868FB
:1017B0004901014319601D4B1A6083222260196898
:1017C0001B4B186802F004F8311C000902F000F805
:1017D0001849030A184A0B60C0B203231060236043
:1017E000164B1D60164B186860201C680440602C66
:1017F000FBD101E0146800E001201C680442F9D12B
:10180000044B01221A700F4B802292031A600523A9
:101810000B6070BDE002001004E100E0A440044051
:101820000C800040A8400440808004409880044020
:10183000AC0400100480004000800040088000409C
:101840001480004000E100E000B5044A2023116844
:101850001942FCD0024B186000BDC0461480004005
:101860000080004008B5FFF77BFF0023437308BDED
:1018700008B5FFF775FFC27B031C8218107CDA7B6A
:101880007F2101320A40DA735A7B013AD2B25A738D
:1018900008BD10B5041CFFF763FF837B7F22C318CC
:1018A0001C74837B013313408373437B0133DBB2AE
:1018B000437310BD08B5FFF753FF407B431E9841AB
:1018C00008BD30B5002402E00570013401301D5D13
:1018D000002DF9D1121B131C02E00170013B0130F5
:1018E000002BFADCD043C0170240A01830BDF8B579
:1018F000051C0F1C1E1C541E092B01D800240FE0D0
:10190000181C0A2101F064FF221C031C391C281C2E
:10191000FFF7EDFF041C2D1805E02F700134013591
:10192000013A002AF9DC301C0A2101F095FF303120
:101930002970601CF8BDF8B50C1CD9175F18061C7F
:101940004F40551E092F12D9381C0A21002B03DAEB
:1019500001F03EFF434202E001F03AFF031C211C6C
:101960002A1C301CFFF7E7FF041C351813E0002B7E
:1019700000DA951E002201E0B4540132A91A0029B0
:10198000FADCEC43E4172C403519002B03DA2D2345
:101990002B7001340135381C0A2101F05DFF303114
:1019A0002970601CF8BD73B5069E041C1D1C30090F
:1019B000531E00280AD000901A1C201C2B1CFFF775
:1019C000F2FF241805E0217001300134013A002AA9
:1019D000F9DC0F231E40092E01D8303604E0002D1B
:1019E00001D0373600E057362670013076BDF0B5AD
:1019F00085B0041C0F1C002801D0002101700025B7
:101A00006BE0252903D021700132013405E05178C3
:101A1000252904D121700232013401355DE03029DD
:101A200003D001320292202101E002320292029E92
:101A30009C4632782D3A50424241B6180296002216
:101A400005E00A235A438218303AD2B20136307880
:101A5000031C303B092BF4D90296AE186346BE42F4
:101A600001D97A1BD2B269280ED006D863282CD0AF
:101A7000642809D058283ED119E075280AD0782862
:101A80000FD0732837D11AE01E1D201C1B68FFF7EA
:101A900052FF04E01E1D201C1B68FFF728FF331CAB
:101AA00017E01E1D1B68201C0093002304E01E1D70
:101AB0001B68201C00930123FFF775FFEFE71E1D35
:101AC000201C1B68FFF7FDFEE9E71A680120227061
:101AD0000433029A241801322D181178BD4201D224
:101AE00000298ED10023BD4201D2237005E0013CC4
:101AF0002370013D01E001256D4205B0281CF0BDB9
:101B000010B50C1C131C6421221CFFF770FF10BDC4
:101B100000B5031C9BB00A1C01A8191CFFF7F0FFBD
:101B2000632800DDFEE701A800F0A6F81BB000BDA9
:101B30000FB407B504A901C90191FFF7E9FF03B08C
:101B400008BC04B018470EB403B503AA02CA019238
:101B5000FFF7D6FF02B008BC03B0184770B50323E7
:101B6000041C184205D10D1C041C194201D19342DA
:101B700001D3002311E0131C40CD043B40C4032BD0
:101B8000FAD8141FA4080134A400032309191A4029
:101B90000419EEE7CD5CE55401339342FAD170BDF0
:101BA00030B50B040D061D430D430B021D430323EB
:101BB000041C93420DD218420BD1131C043B20C4C9
:101BC000032BFBD8141FA4080134A40003231A40DC
:101BD0000419002301E0E15401339342FBD130BDED
:101BE00000B5002300E00133C25C002AFBD1181CC1
:101BF00000BD00B5031C01E0013101330A781A7001
:101C0000002AF9D100BD30B5031C002406E01D5D9B
:101C1000085D281A05D10134002D02D09442F6D176
:101C2000002030BD00B502E00130002B06D00A785C
:101C3000037801319342F7D0981A00E0181C00BDD8
:101C400008B5FFF769F90B4BFA211868890001F014
:101C50000DFEFFF779FCFFF79DFAFFF74DFB96208D
:101C60000002FFF781FDFEF73BFEFEF727FEFFF7C0
:101C700083FA08BDAC04001010B5041C02E0013466
:101C8000FFF7E2FD20780028F9D110BD30B5F82328
:101C90008A01DB0013404A05920E1343F822120218
:101CA000114019430A235943CA1083181C1CEB34F2
:101CB0005D782478EA336C401B7824021C43835CF3
:101CC000201C58400723194008418005800D30BD75
:101CD00008B5054B011C984201DD044BC1180448AE
:101CE000EA38FFF7D3FF08BDFF17000000F8FFFF39
:101CF000EC40000008B54018511A013101F018FEFF
:101D000008BD08B5801889189A1A0132FFF726FF16
:101D100008BD000010B5CB00591A074B0F22C91897
:101D20000023CC5C14400470CC5C01332409447063
:101D30000230072BF5D110BD4C05001010B5CB00BB
:101D4000591A064BC918002342780478120122431D
:101D5000CA5401330230072BF6D110BD4C050010D8
:101D600030B5B14B87B0D96EB04D4A1E91416A462D
:101D7000D175A96A1A1CC806400F0138062807D871
:101D800001F012FD040C1F1217191C00022409E0B7
:101D90005A6E16329200D3581C1C15E05B6E163337
:101DA0009B00D45800230FE09B6DD46DA3420ADC46
:101DB0000AE0022403E00C24032305E00D24231C85
:101DC00002E00D24EEE70D242C6148111F2800D9F4
:101DD00022E16A461732944901F0F0FC200022000B
:101DE00028002A002D002F00380040004400490040
:101DF00051005F0067006F00770085009300A2002C
:101E0000B400C300D500D300E300E600E900F10010
:101E1000010105010F01110113011901081C00E066
:101E20008348191C221CFFF765FFF5E08148F8E79D
:101E30000A1C0E3203E07E4809E00A1C1C32081C12
:101E4000111C1A1C231C01F0F9F8E5E07948011C6B
:101E50000E391A1C231CFFF754FFDDE07448011CE7
:101E60000E31EEE70A1C1C32081C111CF1E70A6E49
:101E70001020002A00D00A200A1C0E3206E00A6E4A
:101E80001020002A00D00A200A1C1C3200946C4644
:101E9000173402900194081C51E001201070086E64
:101EA0001022002844D00A2242E00A6E1020002AA4
:101EB00000D00A200A1C0E320EE001201070086EBD
:101EC0001022002855D00A2253E00A6E1020002A62
:101ED00000D00A200A1C1C3200946C461734029071
:101EE0000194081C78E00A6E1021002A00D00A2113
:101EF000504A68461730019002910094101C111C42
:101F00001DE00A6E1020002A00D00A20494A0094E1
:101F10006C46111C173402901C390194101C0EE001
:101F2000096E012010701022002900D00A224149B8
:101F300068461730019002920094081C002201F0BC
:101F400087F869E00A6E1020002A00D00A20394A7A
:101F500000946C46111C173402901C390194101C1B
:101F60003AE0096E012010701022002900D00A22E8
:101F7000304968461730019002920094081C0022F4
:101F80002AE0012010700A6E1021002A00D00A21D8
:101F9000284A68461730019002910094101C0021D5
:101FA0001AE0009222481CE00092224819E00A6ED2
:101FB0001020002A00D00A200A1C1C3206E00A6EFB
:101FC0001020002A00D00A200A1C0E3200946C4611
:101FD000173402900194002001F063F81CE0009295
:101FE000081C002104E00D1C1C35081C0092291C53
:101FF0001A1C231C01F0B0F80EE0081C02E00C488B
:1020000000E00C48191C221C01F0BFF804E0081C79
:10201000221C191C01F0C4F86B46DA7D024B07B094
:102020000120DA6630BDC046B00400104C0C001030
:10203000BE040010CC04001010B506490B1C8833F8
:102040001A68141C1E34A4006050013203210A4097
:102050001A6010BDB0040010054B0320191C883114
:102060000A68013A02400A601E329200D058704756
:10207000B0040010F8B5114D2C1C8C3420680130D0
:10208000FFF726FE0E4B0122D8629F6AAB6E061C3C
:1020900002409A4210D1830703D420680230FFF730
:1020A000CBFFFF239B001E40B601BF10044B8C35B5
:1020B000374301222F60DA600220F8BDB00400101F
:1020C0004C0C001030B50C4B0C489A6A031C8C3336
:1020D0001C68D3059B0E910500D5403B856E921080
:1020E00001210A40AA4204D1E3188C300360024B5C
:1020F000D960012030BDC0464C0C0010B004001067
:1021000008B5084B5A1CD07F9A1CD27F00011202DE
:102110001043DA7F0333DB7F10431B031843FFF7C1
:102120008BFF08BDB004001038B5FFF795FF0649D6
:1021300003230F22051C5C1815400133257700117D
:10214000072BF7D138BDC046B004001008B5FFF723
:1021500083FF034B01228C331860024BDA6008BD09
:10216000B00400104C0C001010B5064CA36E002BF0
:1021700006D0FFF771FF044B8C3401222060DA6037
:1021800010BDC046B00400104C0C001010B5064C39
:10219000A36E002B06D1FFF75FFF044B8C340122A6
:1021A0002060DA6010BDC046B00400104C0C001076
:1021B00008B5124B1B68002B00D09847104B5A698A
:1021C000002A15DD012A07D1DA69002A04D09A61B4
:1021D0000022DA610A225A615B690322191C9143C9
:1021E0000A1E02D0074A0121D166054A013B53610C
:1021F000044B90331A68024B5A6208BD70030010FA
:102200004C0C0010B004001000B5064B5A69002AAF
:1022100007DD9A690F21044B1140D9771211013360
:10222000DA7700BD4C0C0010B0040010044B597F4D
:102230009A7F090112020A43197F0A435A677047BD
:10224000B004001030B50B1C093B012B0FD8084A15
:1022500000239C18257FC45CA54205D0054B083996
:102260005A681143596002E001330E2BF1D130BDA1
:10227000B00400104C0C001008B50E4B1B68292B45
:1022800017D008290DD0192913D1427808231A42F2
:1022900002D00022027002E00F2303700723437074
:1022A00005E000231A1CC25401330E2BFBD1FFF7AB
:1022B00045FD08BD4C0C00101FB50D4B5C6F002890
:1022C00002D00F22944304435C676846211CFFF749
:1022D00021FD6846211CFFF7CFFF054A00236C460D
:1022E000185D9918013308770E2BF8D11FBDC04631
:1022F000B00400101FB5124B0F225C6F94430443CF
:102300005C67104B1B68292B01D0082C17D068463E
:10231000211CFFF7FFFC6846211CFFF793FF084ACA
:1023200000239918097F6846195401330E2BF8D100
:10233000211CFFF7A1FF6846211CFFF7FFFC1FBD12
:10234000B00400104C0C00101FB5114B114C1B6851
:10235000292B02D0636F082B18D0616F6846FFF7F6
:10236000D9FC616F6846FFF76DFF0A4C00231A190C
:10237000127F69465A5401330E2BF8D1616F6846BB
:10238000FFF77AFF616F6846FFF7D8FC1FBDC046B4
:102390004C0C0010B004001010B50D4C631CD87F1D
:1023A000A31CDB7F00011B021843E37F1843E31CDF
:1023B000DB7F1B031843FFF78BFC0F23021C1A4023
:1023C00022770211134000126377A07710BDC04638
:1023D000B0040010044B5A6E16329200D258121AF2
:1023E00051424A41DA667047B004001000B5064B0E
:1023F0005A6E16329200D1580139D150002901DAB3
:102400000D21D15000BDC046B004001000B5064BF0
:102410005A6E16329200D1580131D1500E2901D195
:102420000021D15000BDC046B004001000B5094BDA
:102430005A6E16329200D2580D2A03D11A1C293234
:10244000127805E09A18507F117F0001021C0A43A0
:102450005A6500BDB004001010B5084B0F245A6E29
:1024600016329200D1585A6D581814400131047731
:102470000D2902DC5B1812111A7710BDB004001090
:1024800030B50F4B5A6E596D16329200D2580D2A44
:1024900007D11C1C29342478F020084020435865BB
:1024A00007E09818447F057F24012C435C650B11DD
:1024B0004377034B9A180F231940117730BDC0465C
:1024C000B004001008B504480022011C1C390D237B
:1024D000FFF717FC08BDC046E804001008B5044823
:1024E0000022011C1C310D23FFF70BFC08BDC04668
:1024F000CC04001008B504480022011C1C310D2337
:1025000000F09CFD08BDC046CC04001008B504488E
:102510000022011C0E390D23FFF7F3FB08BDC04656
:10252000DA04001008B504480022011C0E310D2306
:10253000FFF7E7FB08BDC046CC04001008B504480F
:102540000022011C0E310D2300F078FD08BDC046AD
:10255000CC0400100C4A0023111C46310B70111CD6
:1025600047310B70111C48310B70111C49310B7035
:10257000111C4A310B70111C4B310B70111C4C316A
:102580004D320B7013707047B004001000B5074A4D
:10259000011C042300208A1804E0D1184631097870
:1025A00040000843013BF8D200BDC046B004001013
:1025B00030B5074A00238918012206E0CC18051C13
:1025C00046341540257040100133042BF6D130BD40
:1025D000B004001038B50020FFF7D8FF084C051CE8
:1025E0000021207FFFF7E4FF25770420FFF7CEFFCF
:1025F0000421051C607FFFF7DBFF657738BDC0460F
:10260000B004001010B50020FFF7C0FF034C207786
:102610000420FFF7BBFF607710BDC046B004001078
:1026200010B5054C0021207FFFF7C2FF607F042119
:10263000FFF7BEFF10BDC046B004001010B5094C36
:10264000231C8C3318680130FFF742FB064B021C39
:10265000D8620F231A4022770211134000126377C9
:10266000A07710BDB00400104C0C001010B5094C40
:102670000021201C0D22FFF73DFB201C0E30002105
:102680000D22FFF737FB201C1C3000210D22FFF725
:1026900031FB10BDB004001010B50C4B00211A1C0A
:1026A000187F1C7801312043187701330E29F7D1A8
:1026B000936E002B08D0064B1B690D2B04D1137FA2
:1026C000111C29310B70537310BDC046B0040010AB
:1026D0004C0C001010B50C4B00211A1C1C7F1878F4
:1026E00001312040187701330E29F7D1936E002B6A
:1026F00008D0064B1B690D2B04D1137F111C293107
:102700000B70537310BDC046B00400104C0C001089
:102710007FB500230C4A0D251C1C1118097F0130C0
:102720006E469955C60F8542664176420133111CAB
:1027300030400E2BF1D100236C46185DCA180133CE
:1027400010770E2BF8D17FBDB004001010B5074BE9
:102750005A6E16329200D1585C1801392077D15048
:10276000002901DA0D21D15010BDC046B00400107F
:10277000034A0023111C943198320B601360704798
:10278000B0040010034B012194331A684A401A60C8
:102790007047C046B0040010044A002313678C320F
:1027A0001360034B0122DA607047C046B00400108A
:1027B0004C0C001008B59A4B0F20996A994A8B105F
:1027C00018408911013852560E2800D9C1E000F096
:1027D000EBFF08111A2327C02EC0C037C0C0C03B72
:1027E0003F00002A00DAB4E08F4B9A1840320023F1
:1027F0009371A9E0002A00DAABE08B4B01209A1814
:1028000040329071A4E0002A00DAA2E0864B9A18C8
:1028100040329279DA6697E0081CFFF797FF93E061
:10282000002A00DA95E0101CFFF7D4FD8CE0002AA6
:1028300000DA8EE07C4B596E16318900CA5083E075
:10284000081CFFF757FD7FE0081CFFF735FD7BE014
:10285000002A00DA7DE0101CFFF75AFF74E0724B8B
:1028600001209833186073E0FFF7E0FD6CE0FFF79C
:1028700093FF69E0FFF726FE66E0FFF7EDFD63E0FA
:10288000694B00225A665FE0FFF728FE5CE0FFF725
:10289000F7FD59E0644B0120586659E0FFF72AFE26
:1028A00052E0FFF7CBFE022052E0FFF72FFE4BE095
:1028B000FFF726FC48E0FFF735FE45E0FFF7D6FEC0
:1028C00042E0FFF731FC3FE0FFF738FE3CE0FFF766
:1028D0009BFC39E0544B00221A6635E0FFF7A6FC5A
:1028E00032E0514B0120186632E0FFF741FF2BE048
:1028F000FFF72AFD28E0FFF745FF25E0FFF74CFD35
:1029000022E0FFF78DFE1FE0FFF72EFC1CE0FFF733
:10291000C3FE19E0FFF776FE16E0FFF737FC13E081
:10292000FFF7D8FE10E0FFF715FE0DE0FFF740FCC3
:102930000AE0FFF75BFD07E0FFF74CFE04E0FFF75E
:1029400065FD01E0FFF702FC012001E001204042AB
:1029500008BD982BBED03EDC382B9BD01DDC1C2B39
:1029600000D187E70CDC0C2B00D178E702DC002BD0
:10297000EAD0EBE7162B00D176E7182BE6D176E705
:10298000282B00D17CE702DC262BDFD175E72C2B2E
:1029900000D179E7362BD9D179E7662B00D18AE7C8
:1029A0000CDC4C2B00D17CE702DC3C2BCED175E754
:1029B000562B00D179E75C2BC8D179E76C2B00D17D
:1029C0007FE702DC682BC1D178E7762B00D17BE76B
:1029D000882BBBD17BE7E62B00D19BE726DCC82BFD
:1029E00000D188E70CDCA82B00D17AE702DC9C2B15
:1029F000ACD173E7B82B00D177E7BC2BA6D177E732
:102A0000D62B00D17DE703DCCC2B00D09EE775E709
:102A1000D82B00D178E7DC2B00D097E777E7C046CA
:102A20004C0C0010EC540000B0040010F32B00D14B
:102A30007CE70EDCEC2B00D172E703DCE82B00D046
:102A400084E76AE7F12B00D16DE7F22B00D07DE738
:102A50007AE7F62B00D16FE703DCF52B00D075E7A2
:102A600067E7F72B00D16AE7F82B00D06EE769E73C
:102A700038B5184C231C8C331868FFF729F9E26E1F
:102A8000154BA2660022E266DA6003229862251CDA
:102A900010401C1C022809D090420AD0012802D004
:102AA000FFF788FE07E0FFF7E5FA04E0FFF758F9C3
:102AB00001E0FFF707FB002807DDE368002B04D1E6
:102AC0002B1C8C331A6812181A6090352B681B184F
:102AD0002B6038BDB00400104C0C0010034B0122D9
:102AE000DA660F229A775A771A777047B004001087
:102AF00010B5054C0549201C00F01AFFFFF7EEFF4A
:102B00000123636610BDC046B00400109C0700009E
:102B100000B5074B00201B680F2B08D1054B1A7816
:102B2000824204D11868044B1840431E984100BDEE
:102B300080000010B004001000FFFF0038B5164BF5
:102B40001A1C98321268002A04D0144B1D68012305
:102B50001D4001E094331D68114CA3689D4202D1D1
:102B60006268002A16D0002D02D1002B0AD111E094
:102B70000C4B1B68002B02D06168281C984700236F
:102B8000636006E0074B1B68002B02D0281C291C41
:102B90009847A56038BDC046B004001090030010EF
:102BA0004C0C00108803001013B500230093019310
:102BB000244B1B68002B02D0684601A99847224984
:102BC000009B0878214A00280CD0002B02D0022359
:102BD000137035E01378013BDBB21370002B2FD15B
:102BE0000B7009E0002B0CD11378002B28D0013B8F
:102BF000DBB21370002B23D1154A1360154A136002
:102C00001EE014490968581A44426041400010709F
:102C100011484469021C002C04D08B4202D10A23C3
:102C200043610DE000290BD10A21516101999361A3
:102C3000D161084A1360064B02221960034B1A70D7
:102C400013BDC04678030010940300107C030010ED
:102C5000800C00107C0C00104C0C001008B5FFF725
:102C6000A3FF08BD10B5094C20600948016009495F
:102C70000A60094A1360094B029A1A60084B039ACA
:102C80001A60084A084B1A6010BDC046880300103D
:102C900078030010840300108003001074030010F8
:102CA000800000105D2C00007003001008B5084B78
:102CB000084A196812688A1A1A6006D5FA22520060
:102CC0001A60054B1A6801321A60FFF737FF08BD1A
:102CD000840000107403001090030010F7B50E1C60
:102CE0000E21051C019200F023FE1A4B03240C2731
:102CF0009E420FDD09236B7301232B7328E0301CE8
:102D00000A2100F009FE301C29550A2100F0AEFD11
:102D10000134061C002E06D0E30F0022A7425341C7
:102D2000DBB29342EBD1019AA31A033B2B70621BD7
:102D30002B1C01E0195D5973013BD1180229F9D10F
:102D40000F231C1B002301E0013C2B55032CFBDC53
:102D5000F7BDC046FFC99A3B38B50C4B01221A702B
:102D60000B4B02221A700B4D0B4C08E0186888427E
:102D700008D01B682360FFF799FFFFF715FF2B684A
:102D80002168024A10780028F0D138BD9403001061
:102D90007C030010800300108C030010F7B51C4D5D
:102DA0009B235B000E1C1B4AE95C1B4BAC5CEB5C81
:102DB000002902D00F22144002E08021072449009C
:102DC0009A225200AF5C154ACB1AAA5C3435BA1A63
:102DD00080277F00791A009107210C1B01321049CE
:102DE0000194FEF7B0FE00230E4F33704124FF35EF
:102DF000301CFEF7F5FE2A786B783018D31A391C90
:102E0000221C0134FEF79FFE013D462CF0D1F7BD98
:102E1000B0040010370100002F0100003501000050
:102E2000FC5400000955000070B5434B434C1A1C7C
:102E30009432126890B0A061E161002A17D118287D
:102E40000BD1C32909D13E4A12680F2A05D1181C9B
:102E500038300E21162200F0DDF8A369182B04D1BA
:102E6000E369332B01D100F07FF8FFF737FE0A2327
:102E7000314D6361334E01232B678C35FFF7F8FD2D
:102E80002B68B34216D006DC2F4A93420DD02F4A4E
:102E900093423AD11DE02E4A934210D02D4A9342DC
:102EA00020D02D4A934230D10EE0254B1B680A2BCF
:102EB0002BD112E0224B1B680B2B26D10DE0204BAF
:102EC0001B680C2B21D108E01D4B1B680F2B1CD15C
:102ED00003E01B4B1B68102B17D1FFF72FFEFDF7EC
:102EE000F6F812E0164B1B680F2B0ED11B4C236813
:102EF000002B0AD0684608A9FFF750FF23686846F0
:102F000008A998472B6827332B60154B1A68154B77
:102F100010681968884205D012681A60FFF7C6FE6B
:102F2000FFF742FE044B1B6F002BA7D1FFF706FEF5
:102F3000FFF712FF10B070BDB00400104C0C001071
:102F400080000010130D0000070C00006A0C000048
:102F5000990D00003E270000790D00008403001049
:102F6000800300108C03001070B5254C23681D6889
:102F7000FFF7F2FE23681A689542FCD01E68FFF73F
:102F8000ADFD204B0A22204C5A6118229A6115226D
:102F9000DA61231C903300221A60FFF79FFD2D3663
:102FA00001232367FF36164C184D0AE0FFF760FD3A
:102FB00023682A681968914203D01B682B60FFF7C9
:102FC00075FE23681B689E42F0D10F4C1820231C0D
:102FD000903300211D68FFF727FF0D4B281C19684F
:102FE00000F044FC3834011C0422201CFFF776FE5C
:102FF000044B18229A610022281CDA6170BDC04679
:10300000800300104C0C0010B00400108C03001062
:1030100074030010F0B501240DE005780B1C254069
:1030200006E0C65CED0077083D43C554351C2540DD
:10303000013BF6D5013A002AEFDCF0BD30B504E0E3
:10304000845C8D5C85548C5401329A42F8DD30BD2D
:10305000F7B5099D0AAC2678089F2C7894461D1C6C
:10306000002A0DD118E063465B5D4A5DD218131942
:1030700001920024B34201DB9B1B0124435501351F
:10308000BD42F0DD0AE0CA5C12190024B24201DB45
:10309000921B0124C2540133BB42F4DD099B1C7016
:1030A000F7BDF7B5099E0AAC2778089D347800284B
:1030B0002FD000292AD01E1C9446002A0ED1013F91
:1030C00018E063469B5D8A5DD21A131B00240192AF
:1030D000A34201DADB19012483550136AE42F0DD4B
:1030E00037E0CA5C121B0024561C01D13A1C012493
:1030F000C2540133AB42F4DD2BE0D15C49420C1BDE
:10310000211E01D0E1190124C1540133AB42F4DD89
:103110001FE000291BD0181C002A06D10EE00E5C0F
:10312000135C0130F31A1C1BE40FA842F7DD10E01A
:10313000CA5C0133141B013462425441AB42F7DDD7
:1031400007E0D15C013349420C1B611E8C41AB424C
:10315000F7DD099A1470F7BD70B5049D01242C7039
:10316000141C002905D10BE0065D0A5D96420BD1C7
:1031700001349C42F8DD05E0815C002904D1013274
:103180009A42F9DD00232B7070BD00B503E04318AF
:103190005B78435401319142F9DB0023435400BD75
:1031A00000B504E08318013B1B788354013A8A423E
:1031B000F8DC0023835400BDF0B5114B1A785B781E
:1031C000825C1A4000D040220E4C0F49231C261C62
:1031D00004C32C3600221A6001240A1C123117780D
:1031E0005578C75D3D4202D01F6827431F600232F9
:1031F00064008A42F3D10433B342EBD10020F0BD26
:103200007D010010140E0010C900001030B512230B
:103210004B43334A0131D3188A0051181A785C782D
:10322000825C144204D02F4A5F2452189470547068
:103230009A78DC78825C144204D02A4A7C245218A2
:10324000533214701A795C79825C144204D0254A96
:103250007C245218A33214709A79DC79825C14426F
:1032600007D0204C5F226418251CA235A1342A7097
:1032700022701A7A5C7A825C144204D0194A7C2447
:103280005218A03214709A7ADC7A825C144204D00C
:10329000144A7C245218503214701A7B5C7B825C76
:1032A000144207D00F4C5F226418251C523551344C
:1032B0002A7022709A7BDC7B825C144204D0094A1B
:1032C0002E245218A43214701A7C5B7C825C134248
:1032D00004D0044B5918F43127230B70002030BD63
:1032E000C9000010840C0010F8B52D4C071C0025F7
:1032F000201C20214F22FEF753FC002D04D0221C5D
:103300007C23393223701370231C4F330021013585
:1033100019705034052DEBD1214B2D22181C38305B
:103320000270181C37300270A1209A705A70400049
:103330005F221A541B481A54A320400019541A49FA
:1033400008784978385C014204D0191C5331523353
:103350000A701A700024211C381C0134FFF756FF34
:103360000A2CF8D1114D124E00242B786A78FB5CA0
:103370001A4201D0315905E03059FEF731FC0D49B0
:10338000091A0A310C48043400F0DCFA0235242C06
:10339000EBD10A49084800F0D5FA0520F8BDC0462F
:1033A000840C0010410100007D0100108800001015
:1033B0009C0000107F010010C40D0010115500008A
:1033C000F0B585B001900027FDF778FA6A4C3E1CF5
:1033D0006A4A7542754113687D19012B05D1684809
:1033E0000D210C22FDF72AFB02E0002B00D1CDE0DD
:1033F000002303AA537023687F210B405C2B00D16C
:1034000098E02ADC382B00D18EE013DC072B6AD041
:1034100006DC022B00D193E0062B00D0B6E041E0A1
:10342000212B00D184E0232B00D187E01C2B00D07E
:10343000ACE081E04F2B4ED007DC3F2B62D0402B1D
:1034400062D0392B00D0A1E064E0542B76D05B2B06
:103450003FD0502B00D099E06AE0732B66D010DC8F
:10346000662B3AD005DC5E2B56D0622B00D08DE067
:1034700062E06F2B3BD0712B52D06D2B00D085E0DA
:103480002DE0792B4AD006DC762B4BD0772B3DD024
:10349000742B7BD146E07D2B23D07F2B25D07C2B3A
:1034A00074D135E031231370022E4BDD231C083B11
:1034B0001B681940542908D0032E43D0231C0C3B11
:1034C0001A687F231340542B3CD14C2203AB1A7053
:1034D00038E0322335E0332333E0342331E0352341
:1034E0002FE036232DE037232BE0382329E0392342
:1034F0001370062E26DD231F1B681940472323293E
:1035000020D11EE030231CE02D231AE0412318E0D7
:10351000422316E0432314E0442312E0452310E045
:1035200046230EE048230CE04C230AE0502308E039
:10353000522306E04F2304E0552302E04E2300E02F
:1035400049231370ADB203A8291C0022FDF7ECFA41
:1035500023681A0605D5E91D89B20A480022FDF73D
:10356000E3FA2368DA0572D50735A9B206480022C6
:10357000FDF7DAFA6BE0C046140E00108C01001063
:10358000A73B00007C400000195500002368012281
:10359000134206D0A818C0B2002107220223FDF76B
:1035A0002DFA23680222134205D0A81DC0B20021C3
:1035B0000623FDF723FA236804210B4205D0A81D3A
:1035C000C0B202220623FDF719FA236808210B4234
:1035D00005D0681CC0B207220223FDF70FFA23684A
:1035E000DA0606D5681CC0B2042102220623FDF7C4
:1035F00005FA23689A0606D5681CC0B2002102228B
:103600000623FDF7FBF923685A0606D5681CC0B2ED
:10361000042107220223FDF7F1F923681A0607D5D2
:10362000281C09300222C0B20821131CFDF7E6F95C
:103630002368DA050BD5EDB2281C0930C0B20B2186
:103640000A35FDF7C5F9E8B20A21FDF7C1F90136DF
:1036500004340C370B2E00D0BAE61B480321062297
:10366000FDF7ECF9194D1A4E1A4F0024019A2B78E8
:10367000D35C6A781A4205D0A3009859395D0922B3
:10368000FDF752FA01340235092CEFD1FFF740FA69
:10369000002814D006240321201C00F0E7F80321A1
:1036A000C5B2201C00F038F9281CC9B2FDF790F90A
:1036B000092C01D10B24EEE701340E2CEBDDFDF7D4
:1036C00007F905B0F0BDC046623A0000880000105E
:1036D00090010010C000001070B5041CFFF76CFDD5
:1036E000201CFFF76DFE0A4B1B78002B0ED0201C10
:1036F000FFF7FAFD074CC8235B00074EE518211CB5
:10370000301C5034FEF714FAAC42F8D1002070BDE2
:1037100095030010840C00103D3A000000B589B0FC
:1037200000280ED0FDF7A9F801A80921FEF7F2FA4A
:10373000684612300A21FEF7EDFA01A8FFF7CCFF28
:1037400008E0FDF7A2F8044B1B78002B02D00348D9
:10375000FEF7EEF909B000BD950300101B550000FF
:1037600000B5FEE700B5FEE708B50A4B0A4A0B496B
:1037700003E010780132187001338B42F9D3084B03
:103780000849002201E01A7001338B42FBD3FCF799
:1037900011FEFEE70000001072550000B401001099
:1037A000B4010010400E001002B4714649084900EF
:1037B000095C49008E4402BC7047C04603B47146A0
:1037C000490840004900095A49008E4403BC70472B
:1037D000002934D00123002210B488422CD30124C4
:1037E0002407A14204D2814202D209011B01F8E759
:1037F000E400A14204D2814202D249005B00F8E712
:10380000884201D3401A1A434C08A04202D3001B3D
:103810005C0822438C08A04202D3001B9C08224370
:10382000CC08A04202D3001BDC082243002803D0AE
:103830001B0901D00909E3E7101C10BC70470028E0
:1038400001D00020C04307B4024802A140180290F2
:1038500003BDC046D90000000029F0D003B5FFF732
:10386000B9FF0EBC4243891A1847C046002941D00F
:1038700010B4041C4C40A44601230022002900D5AA
:103880004942002800D5404288422CD30124240715
:10389000A14204D2814202D209011B01F8E7E400EF
:1038A000A14204D2814202D249005B00F8E788427B
:1038B00001D3401A1A434C08A04202D3001B5C08F3
:1038C00022438C08A04202D3001B9C082243CC0850
:1038D000A04202D3001BDC082243002803D01B09AE
:1038E00001D00909E3E7101C6446002C00D54042D2
:1038F00010BC7047002806D003DB0020C0434008FE
:1039000001E08020000607B4024802A1401802909E
:1039100003BDC046190000000029EBD003B5FFF736
:10392000A7FF0EBC4243891A1847C0467047C046DD
:1039300000B5002905D000230139037001300029AA
:10394000FAD100BDF8B5041CA30719D1231C04CB80
:103950000F4D104E50199043021C201C32420FD1C3
:10396000181C0B4F04CBD5199543354208D1181CB0
:10397000074F04CBD51995433542F1D000E0013013
:103980000378002BFBD1FEF734F9201CF8BDC046AC
:10399000FFFEFEFE8080808053455249414C20430B
:1039A0004F4E534F4C450025732072656164790D6D
:1039B0000A00444D31304343000D0A4279652E2EF2
:1039C0002E0D0A002573202573202025694D485AA5
:1039D00000563700202025692E25303369560042D5
:1039E00041543A2025696D560D0A002578000D0ACC
:1039F000253032782020000D0A413A200020202571
:103A0000633A20000D0A4D3A20002020473A202535
:103A10003032780D0A0057616974696E6720666FED
:103A20007220646174612E2E2E0D0A0042616420A2
:103A30006D6F64656C0D0A00526561642025730D1D
:103A40000A004F4B004641494C4544006F6E006FE1
:103A50006666004C43442064656275672025730DDB
:103A60000A0003030000000303005C0003030C00D2
:103A70000C03037C287C03037C447C030324104850
:103A800003032854080303000C0003033844000315
:103A90000344380003032010080303103810030305
:103AA00080400003031010100303004000030320B4
:103AB000100803033844380303007C0003036454F4
:103AC00048030344542803031C107C03034C542470
:103AD0000303385420030304740C030328542803FD
:103AE000030854380303005000030380500003030D
:103AF0001028440303282828030344281003030440
:103B000054080303384C5C030378147803037C5493
:103B100028030338444403037C443803037C54449F
:103B200003037C1404030338443403037C107C0334
:103B300003007C00030320403C03037C106C030360
:103B40007C404003037C087C03037C047C03037CEF
:103B5000447C03037C1408030338447803037C1477
:103B60006803034854240303047C0403037C407C5F
:103B700003033C403C03037C207C03036C106C0378
:103B8000031C601C030364544C03037C44000303C4
:103B90000810200303447C00030308040803038087
:103BA000808003030408000007080400000000BF31
:103BB00001BF010905000007000700070007130AFD
:103BC00000002000E400FC003F00E700FC003F0094
:103BD0002700040F0800000C011E01FF03FF032251
:103BE00001E201C2190D00000E001F001101910138
:103BF000FF007E00FC00FE0113011101F001E01442
:103C00000A0000EE00FF0111011101BF01EE00E00A
:103C10000130011001050300000F000F0A0500002C
:103C2000F800FE03070701040B0600000000010472
:103C30000707FE03F80F08000000000A000E001F2F
:103C4000001F000E000A11090000100010001000F3
:103C5000FE00FE00100010001008040000000480A8
:103C60000780030D07000010001000100010001066
:103C70000010080400000000800180010D07000C06
:103C8000000FC003F0003C000F00030F080000FE0F
:103C900000FF01010101010101FF01FE1008000008
:103CA000000002010201FF01FF01000100011008F4
:103CB00000008601C7016101210131011F010E01D0
:103CC0000F08000082008301110111011101FF01A1
:103CD000EE11090000300038002C002600FF01FF23
:103CE000012000200F08000080009F011F0111012A
:103CF0001101F101E10F080000FC00FE010B0109B8
:103D0000010901F901F00F08000001000100C101E3
:103D1000F1013D000F00030F080000EE00FF01114C
:103D20000111011101FF01EE0F0800001E003F010B
:103D300021012101A101FF007E0804000000008C88
:103D4000018C010804000000048C078C0312090098
:103D500000200070005000D80088008C010401048D
:103D60000111090000480048004800480048004888
:103D70000048004811090000040104018C0188007A
:103D8000D80050007000200D07000002000300B1B1
:103D900001B9010F0006190D0000F800FC0106032F
:103DA000FB06FD0505050505FD05FF050601FC01F2
:103DB000F8120900008001F0017C004F004F007CE8
:103DC00000F00180010F080000FF01FF0111011147
:103DD000011F01FE01E0110900007C00FE008301CB
:103DE00001010101010183018211090000FF01FFAE
:103DF000010101010101018301FE007C10080000A6
:103E0000FF01FF01110111011101110111010F0841
:103E10000000FF01FF01110011001100110001124B
:103E20000900007C00FE008301010121012101E362
:103E300001E20112090000FF01FF01100010001053
:103E4000001000FF01FF010A0500000101FF01FF52
:103E50000101010B060001000101010101FF01FF49
:103E600010080000FF01FF0138006C00C60083014C
:103E7000010110080000FF01FF0100010001000125
:103E800000010001160B0000FF01FF010F003C00C4
:103E9000F000F0003C000F00FF01FF0112090000DC
:103EA000FF01FF010F001C007000E001FF01FF0196
:103EB000130A00007C00FE008301010101010101E1
:103EC0008301FE007C0F080000FF01FF012100219B
:103ED0000021003F001E140A00007C00FE00830148
:103EE0000101010101038307FE047C0412090000A3
:103EF000FF01FF01210021007100DF008E010001A0
:103F0000110900008E009F01110111011101110121
:103F1000F301E211090000010001000100FF01FFAF
:103F2000010100010001110900007F00FF00800174
:103F3000000100018001FF007F1109000007001F40
:103F4000007800E001E00178001F0007190D000073
:103F50000F007F00F001E0017C001F001F007C00CB
:103F6000E001F0017F000F120900008301C7016C1E
:103F700000380038006C00C70183011109000001FE
:103F80000007001E00F801F8011E000700011209D9
:103F900000008101C1016101310119010D01070119
:103FA000030100070008000A01001811101338313E
:103FB000303378717073C8C1C0C3888180838484B2
:103FC0008782C5C4C7C27574777235343732151409
:103FD0001712020702080201000301090304020488
:103FE0000205030500062024282C383C4044484C98
:103FF0004669726D776172652025735F56370D0AC9
:1040000000252D3130732025732573000D0A547956
:10401000706520273C636F6D6D616E643E203F27A5
:1040200020666F7220706172616D730D0A005570A9
:1040300074696D65202575730D0A003F0025730DA9
:104040000A0D0A00564F5941474552203E3E200076
:1040500025630048656C70004E6F20706172616D61
:1040600073004B6579207072657373003C6B6579E2
:10407000313E203C6B6579323E202E2E2E00447559
:104080006D70206D656D6F7279006C004C6F6164AE
:10409000206D656D6F7279007400546F67676C6591
:1040A00020646973706C6179206F75747075742009
:1040B000746F20636F6E736F6C6500620052656190
:1040C00064206261747465727920766F6C746167C4
:1040D0006500000000800150008002500080035005
:1040E000FC3F0150FC3F0250FC3F03502AA4A7496B
:1040F000BCC10379FD59A29261FE312FA0EE7DEF84
:10410000777DAB8068BD31E024242CDE6EA10BFCF2
:1041100079D7F4E4C86C148AC6606DCD6D50CD0AB1
:10412000C2D71FEC8FFC0DFD3D8D652FB570CC4BBC
:10413000A3966CFEB50672CE24A583504E48256D1D
:104140006EC9664EAE297DE924F8C98B78ADF52796
:1041500048860554143CB4FDED6A5872603C27C291
:1041600061013FD5660E2B020C6554D1FC5A437990
:10417000A853D1E61FAE06C511C22FD3E3DD433DE0
:104180007156FAA19D7E62026555A44B19952AE1EC
:104190005A9080E4E02DF4ED41E16DE39F93A26A33
:1041A0000B5F1C6424CC5C9065496818E75D7082E5
:1041B000179FAEC6414D13F63B7BA6B403BC4EE041
:1041C00001D569E088582D875FA29C20D638E42964
:1041D0008843FC9F09D5F39CF34A29863B7B7D5895
:1041E000F44CF504BC7646BDBC7696BA8B0886B115
:1041F000F9D8254907BBE667289901EF3558094FDB
:10420000582AC6874B556953819A24774BCBE11EB8
:104210008D38353BEDC7A5D21C3B1897B8FFAD2BA9
:10422000728277BE819160A0476D5FD388D4E364CA
:1042300061093CD85BD2F32394B160CE3649E720C4
:104240003C3DF4665B7EFCDFF3CA8FC15B334AAE54
:10425000A1E407FDB3645483D27F5B9569E3D06E1C
:1042600015DE90D4A4FB41DB530792524EB9819ADC
:1042700026020B81F7CC903513551B8CBF19D02C1F
:10428000F27110D7FFBA0B52C6D483A78224E5FC83
:10429000D810A6C9DD606F4B78CEB7971E7808CBD3
:1042A0008950B078B0EC07BD0ACDC160E39294FDAF
:1042B0000787E5DF1728603F34493F41BBDB29B45E
:1042C000D1002F78A906E20B4D71D64A1071F8562D
:1042D00019F65AC237E30C68C5100BC4CA82CB9BCF
:1042E00023DF4A740793499C094EB818CA398A23B8
:1042F000F7B8AE06285FDFC9BC09E5F9E0237DB752
:104300006533A03D14961E91BD91D38683FF86FC34
:10431000C29B17546E07ADBA350E43563CA05B5591
:10432000C4C9F841F1976A53DFE128D7A25BDA5E8E
:10433000897F42CB58A9D3F5596181670A36B4C247
:10434000ACB65B5449DD6DE780A88CDC018674381F
:1043500043D2D0B18A9DE7AA9DA28524FF99970CEC
:10436000B33BC7275AB49D05A1AC5C585E33359A60
:104370007D58F78A13FE84FC2289B20FD629595042
:104380005A9FBADF331BE3C90DF3F89054F6297036
:1043900087771A716AADA54CECCDF6B1E13CC7CD7B
:1043A000D3C232A23565999A396FBA058B69113734
:1043B0006058BE32C40D2D214354A7B7BAC0E7726E
:1043C0003753FB5C929D01590CA6272258BCB68F2F
:1043D0005CAC096FF73B42FFC535EDB46EAE69B515
:1043E00044703722F6B574672F810D9B7C35289E6B
:1043F0003E07D4B79182B507D67C8FA6A348AEE519
:10440000299179B6CA573F30F535D48696D93C17ED
:104410007DD75C58A48E3602BF04B3630E23DEA59D
:1044200066AD822BAD2B36D5A0C1A2375422FE3704
:104430003E88A250216A9AA7963E8067DDE6111554
:10444000D26E6A1EF4CAE4888797FB06708962837D
:10445000A31601D3F00921E306B369E2E30ADEDE25
:104460007C04844F8A6A5931177D59360F34BD1F39
:10447000D3A5CDF3FB9DDCE0616CFF855F796947D7
:104480002625C3CDD53DE5A3EC4E1266268693C9FD
:104490005822505FB102B548B9AD6B664AC2FCEC18
:1044A000E90CAD6538A0BC93675F23AB90DC49B7DE
:1044B0002DD54FB6F42A84A408F130BC79DFF53F3E
:1044C000598FAE9858BB526A69B3344B72B24BF6EF
:1044D000FDD22B81A329D7245E1032C72C7F97B33E
:1044E0008BFAD0E095278C19E009291A3A2E0B9304
:1044F0009A7B159A5B85B59770A7C1C4FD54D18E80
:10450000D59993ADB2A4D538962D6644B2C89327F9
:104510009B951800A497DDE4D908566A63A92594F1
:1045200074C9B13EA4F7C9F9A05B6ADF2EAB963718
:104530002999D38116677A283E181A583ABDEB0B91
:10454000AEC84873CD15180E1CBC4298846F439FAB
:1045500020F72CCC7682132FA8B04BA9C919C5819E
:10456000EC10A87928FDE3E8D45145D54FC42222A8
:1045700009CDC34EBDDC9DD78F5540EE455B3E1542
:10458000B281B15119AA7BF3EC560608AEBAA1BAB2
:104590009FE501D754BD97BC2BD213CB74BB96EAD1
:1045A00024D28A99E6827B1296FF4B8EA258658BA5
:1045B00087AE6BBAB055FB74C8E7B172EAF01DD391
:1045C0002DD19C841753086091A3F5FA9D48F746B6
:1045D0008CA48953A178044FDBEB5A1A123AE26893
:1045E000B42BD0BD99CB453A33E348A24F51212398
:1045F000ECFE654D70834199D5BE128D28CF99B7D9
:10460000C5D4190FE9149E7B2D0814A29010A7A4FD
:1046100052FFAB256E1F66FA5A078C57D08D25A71F
:1046200078CD366200F6020CFB59A161446FF31697
:10463000821D3AD683984CBBE0F195E8CDBCF3C21D
:104640003EA2B3D45D0DDDB6F5A388C80519CFDC55
:1046500013B2CF1A69B8C402A25DC1BEF2CDBA527C
:10466000863A9F77752275443B0DE281628B95B93E
:10467000C2C4882A9D6D645471805240F8C703ED0E
:1046800096B24B2085A0218D7496A5E536D9238658
:104690002E1E569BB5B6699AA1A23D00EF084D6447
:1046A000A71B08E7B279F634AEACE1921F14C275CD
:1046B000B68F90F8D0C43D2B40404FA686B03E2F19
:1046C000C7771F4D2A944A50F2579B096EBBE80BDF
:1046D000444C952244224F8583AE60F1B8ED83624D
:1046E00078BBB7DEACD4A0DB2A9726981AAF2F0987
:1046F0007E084BA5A102FEF173AA32BC84C35BEC19
:10470000E5435F6CB887949222B8F8A7D66A1C94E8
:10471000B2CF1FAF2F016A6BEF8CABBFFFF0B99C1C
:10472000430703EA91FB0E5790E43AB86A5499554F
:1047300095B4746C0D9186028A05FBA1FE5098B564
:104740004842109CC7000004A3D50ECBB4990FD9E2
:104750006D24182AE48D8228862542DB9E7D8D3DBE
:10476000A751969BD2FABBD9136F796242C6E5A6D0
:104770002EC148168D2431C5823A5702EF57E6F90B
:104780002D4AF31485598925FE04554E8799707C6E
:1047900056C76AADD6F23916C961ED4EAC79C92259
:1047A0002D494A2D7E62D22FA03F5C181E595969AF
:1047B00042593647024D76B980E14F51B212FDAFF2
:1047C00052B9B25D00C77A7D00BD56BD24116A148E
:1047D000104795DD83C17CFEE3187B148FE9DC066E
:1047E00040957C8B16B2B423F453EB9ADCE499F138
:1047F000157D1EC5F8A7F64E7F8EA798F21B4DC0FB
:104800006162281C2BD6D92789C0A3498FFAED797C
:10481000937C8ABC8B586EC46B9D94EBA21849257F
:10482000C1A0FAF3C7C4EA1FA94B86DA41DCBA0C6F
:10483000BEF663F6D13746A8CDDFD54E1980BD2B25
:10484000434A8C0F7403FA221A73C751D72E49D6E4
:10485000B5E48B61F04A648ACE9EAF6E4F6AB7A50D
:10486000BCFE22A31A0A2EC73C3FA163DF00873F8C
:10487000A04791B19A47A4913DE517F21D0690EE2D
:1048800087F628351BD2977CD8E55D122BAD2F52C9
:10489000AB4EA0400F1A2D905C75A0B91D438EC67B
:1048A000B32219A7C33EB358CD2E38249BE7C04E80
:1048B000F7A470035CEEAE01A51BEAA5B56B62C55B
:1048C000E439B0515ED3CD966C2704810C6B5882CD
:1048D00054D01859E498D92680B5BDFFD13C1B9718
:1048E00086A36EE1B3C8A60FD5D0D890698268DAE6
:1048F000EB38215C202384081D099E56059F6BD947
:10490000532C7726E56AA288D38785D5CA90C7E35A
:10491000C243B7B8BD1E3C477F197A05F7F1BE17F1
:104920001A0B9C9CF80029A0293CCF5BA20536C538
:10493000AB8D0B62CF55B4A74C1CB9BBA66CEC7BFE
:104940000A00AC4E366B6899947D17EDA599D88B0B
:1049500093DC2CA6C4551EBC0680964DCB717821E5
:10496000E4931052DAD41B0AA9525EA363A531F373
:10497000DF0C1BE55E22DA2804B108A941CC16E160
:10498000B6967A74B5ED5917922CC22ED86193F36E
:10499000B38B35C0A081D1B2CE83F7827479670F13
:1049A000209839DA5EA352B7E02C8F970CF0D1F142
:1049B000CED83C4E12466AE21E5B52CC2877E4A960
:1049C000C2AE683508FDF53EEC914A800EA7048E14
:1049D0006BA0CFA15BEEBBAE6E5628EC2B9B9C531D
:1049E000F08857F104D4869F5B403A3783155D7396
:1049F0002331832785C68640D4B0C944C701BF1878
:104A0000CFE5237B6CD191C00C8533C233F3DF1D1E
:104A1000275D79F7CB5791851CD20BAEC472CC932E
:104A200037C85C03A8FF82FEFF74E800EFC22A28A3
:104A30000A176D7BE7ED1B002353ABE2B096679C32
:104A4000DF6D269BCA4ACA7FBD3067B86142D3D4A6
:104A5000C373443488830510B41C371823576C2F54
:104A60009E18C0B12CB2B12410A5FEA6853A0B2B1E
:104A70006017B871C86A83C30D4F9ADCB8C702C10A
:104A80001E03E69F8489928F17D529B2C19CFF49E6
:104A9000CE2EF310E3A11A50B111CA2026CEF08217
:104AA000DADA1E3B44A94E2A2498054DDFFE0DF8A4
:104AB00095908CBC65B0837546848B7FA094581507
:104AC00090AA505609684F9A0B63330C5612789788
:104AD0000E301AAA78F8ABED651F83B490FCB629A6
:104AE0003255AC8AF84E8B1DCF14E8E59AF55CEE92
:104AF00096A24D852A964EDA69202E3B0B88CAFF76
:104B0000CDE5BC1445B2FE9DDCC1D1516728A5AFEF
:104B1000401E6FFB103B9E4AD9EE0696658EE99CBF
:104B20000B7D3BDDC807BAE09F76D47CA217BA4064
:104B3000EF4C531064B86F9AE217C22258AC6091E0
:104B4000A67EF41E122C23DF559E204640BE9E6496
:104B500001749D354797CB2BA13C5F3A0CDDD3BA4E
:104B6000664EAA740BB0385A2DE748A489187C2DDC
:104B70008D8C119B32335815514DF62CA72F636E37
:104B8000D75447239FBD1D409C92FD7BA7570B7CAC
:104B90004824659D08012574E500AD9CBDBEAE9519
:104BA0006992E571C161289C1BBBD651D84B7F38F7
:104BB0003E5AA0D32534B7943FB5AC3020A16D3B0D
:104BC0006BA9CF387BA44E6EFA81B27A08C4884DA7
:104BD000B54F5068E8269EEBC9E1953A4F41D004A5
:104BE000E1D628282B6170B028D878FE3C8AF2B133
:104BF00070952C7148B85CFFB2A8C74E807F0167E2
:104C0000AD2B09E81B6F0FBC1C42A79DAB9EFCC3DC
:104C100063DF93EE3D57A135A5A42669AB4C277EF3
:104C2000EA8D6C3607A6D7CE1281AEE9BA9EF29213
:104C300064E6179B3171D8DFAB9BEFCAA774C6BC83
:104C40006B85E8ACA406C0D25304A81E4F57AC50E5
:104C50007F45AD0D44D47425C943356E99A84AF2F9
:104C60005896EF4383C4F7C22BBED741B045DD6BE6
:104C7000B67B675D00FEC4FC5C7FCB5C8ED26B674D
:104C8000A941A500705243702D0C629285B6407AFE
:104C9000B408B43D000FE39E74D0F0144F6F1EFEB5
:104CA0007414BE3CC570C16B9DC189C5AD56E0434F
:104CB00059097A61199A23CB9B6A3FE1C938AAAE98
:104CC0009DF8E7F010E3B3EFB05440AEA9FE62DC0C
:104CD0007C2B6AD17DA95BFA1FA39740F9589EAE41
:104CE000D68C8247305538708264AE90BAAE8A65F1
:104CF0003D6D9041AF712B03EFA3F8B631E2ECF4B8
:104D0000A1B6AF82447E8160290FDA8BB99F4560DE
:104D1000B2FEFC0E4377F164C118A6EC111BD1FF63
:104D2000E371E899CEFE894C25274BB5689CA6A572
:104D30004ABDFCAB11821C09CD38232A40074ADE4C
:104D4000D18A4A332994731861BCC0FF7F40B320D5
:104D50006AB57475CC58B3BF6DEF57909D6D40FB2D
:104D60003AF33A6DA87A7B7C07A705F99472C57F60
:104D7000500E6F0563A6B43C79D7FF440D9EFE0824
:104D800069EDC626E3DFE8E89CF0162638A1FEBAF6
:104D9000068B72C999C79D54865DE1C90FE460E92D
:104DA000E3CA9B3644F84F7B0BCC7D68F0BC5121A5
:104DB00092CC6B67462E5A0498269B2E5C1D9D63F1
:104DC00051095CAA8274CBE07C0D3547A68D8DFA23
:104DD000BEF860EA81AE76FEF4B1D363B3A3AB9BB9
:104DE000DEF669589EE0B67FD7144AD7BB89588A49
:104DF0004EA47B6D970BB8A17558368D891D03A302
:104E00001A6E8F14B944EA38D06FC06379236F816A
:104E10005962642352B181A74BE3D6C0259BEFF3BF
:104E20001A81079564E410C84BD49E6EA7A2627ED7
:104E30007278CEF73B5C9FCAF8E60AC07082319B5D
:104E4000433D6E812F1A887E111BEBF936D3EAF3AE
:104E5000F857E9974FFAC10C5330532C5D9D86AC3F
:104E6000B9425413CAC031FA163661EDFE06F99CF8
:104E7000F4639E6D6948104E344C8AFAF254018DE9
:104E80005BA843A3E071BF66FD2AF88BA683740C70
:104E90005A06D3EF1C0F34B9599990CF58AB84EA16
:104EA000CB47004B8BD8BA7BEFA305BBB511ACDA6F
:104EB000E07845EC3B73E214CDC7FD49B6A340D77B
:104EC000A0101E3FAC8D5EADA0A931F08BA2626C2C
:104ED000669F4763523F3A14C5E4B6E48268EA0A23
:104EE000B8A27AB14D2CA6037B46F3818174E240CF
:104EF00054CB3E7E0A600F3D8382E36658EF6E001E
:104F00009A9C18EEE8942192A23A17B18765F45A58
:104F10003B6CA16719808641671CA3B92E4DD86FE1
:104F2000A72B30EABBA19508ACF8388C6F762FDE42
:104F300004F12A2753EB56C7C32348D546D33E274F
:104F4000767F1F9C4F87BE13FD4D92FCD0F922C483
:104F500086944A346C7AC09A4925EFFB8F27040364
:104F60009A3F04E735F4D0C2263F776CAD38F07F26
:104F70007FAF7CC8FA93271E5F4E39E19F6A2DDC14
:104F800004BB75D7286E5AA98C0E68E82FCF091775
:104F90003968F4830F38568ACFDD5E3D41D5FD4632
:104FA000864E25CE38F3E838A95DC3EEDC4D2E8D54
:104FB0000D2A6D79351E7FEF21B368EFF7DDEC39EF
:104FC000DFF37BBFD61E626EBC45A3AA44BA7978D4
:104FD000757CD11E4A3DE879EC48E48AE6EF48B694
:104FE00023EA0DED6FFB4B77D7E29E1B462147B2BC
:104FF00006CCE23E16A690DD1BD2205105AD8D2FCA
:105000000CB1173601E3DEEDF760010ED2ABDEAF77
:1050100037A8147176F48EEF90B87E988CDCC28934
:1050200056C4CF7FE75553D15C72214A10A21F2985
:10503000BC57330A75F607354002B3F0598C88EA3D
:105040007E94A02DEACF55A9ABBDD11DC497346580
:10505000D67AC13DB9622845A185D16F9C5AF4D555
:1050600017DFEA05D182789F2B364B8BC884348AB0
:10507000D0EEB95E080F273158B7F929DBCDC3E769
:1050800061DE216DBE2D55B244E0218B2D77F712E4
:10509000D034F85EDEDAC12F8933168CE0922222FA
:1050A000D10799057F011E3DEC36743592B521FE7E
:1050B000BDCE48BB5BD8F83F209B0E965525444D8E
:1050C0007853E2A65C65A87040163DF10183C136B5
:1050D000C84C59CFF73930ED77D9E53EFCA61FA370
:1050E000672C66D1051D2F5927110B5FB3D6C91543
:1050F00022F7661EFAE813994E10BB69F4B992BE06
:105100002F5512A2B8CB6374310C6E64029BF494D9
:10511000511206DCB9A30EAE7E919E5790540572D3
:10512000ABAC1BBA02F3BEDFF50A6E93BA81285FFF
:10513000ED9CFBB4B0D16247D42F4AA1527D04B29A
:1051400086896C86D97C749138C70AA50A190648E5
:105150008BF5B1AE3D512D151F92B029B140BD3434
:10516000F3A61B6F98CEC583DBABBE262B3949A7B0
:10517000CD0F6AD9C78D494EC5F198B8962EEC1B54
:10518000CB63553717CBE6E3EF1BD889A24482DE09
:10519000382C76814F8F3C4120AC969A7002483271
:1051A0005A06DC41C84D3D17934E0B68AB6260E177
:1051B000A93075B84D1C2190F40E090C81A0176917
:1051C000EDE699D9050098926363FF2BA8596EB755
:1051D000B7427715DAF355ECC8889CB605BB6081F9
:1051E0000FB9871175270D329E0D16F792BFCC248B
:1051F00040A59093F237BF18261121DD3BD1A0C303
:10520000DEA570F2A6B656510D02868A142E737D65
:105210003C466D4FD350ACBA315557E71D19505726
:10522000413E2B2A47ED29E5665A88BDB86F578263
:105230002AA2B27449398519F844BF35538DB9B1E2
:10524000A2B9DD44D2A73E9D922CCBE83641AC4AB0
:10525000CFC073F3F3C61717F03F7571453E8768EB
:1052600083482B51D805749E542A781826BFFEDB3C
:10527000B0FFBF111545E47DE672DB42F641AC7725
:1052800013BDC1BC48D8534844010B7D5D5C9CF8FC
:105290008A7605B55AD168CD5B79E4003795B4DCE0
:1052A000B1A7F84881E4EFB41529E4D8950D75E16C
:1052B000181B2F8FBFBE4A01075C3311B99D1137F0
:1052C0004B6D344E85111E03515FF9E53ED2F82E29
:1052D000ABD79306DCE0B2BC322C68C57595C60B23
:1052E000DF7896301965B04C8B176571D1FEA456E6
:1052F0009510D5C9BDFC162CC6FEE37E7E5092B833
:105300002E593ACC2F7C725F9CD55CC675B5F56E74
:10531000A0D5366F71191EC1971711B95CD9B5099F
:105320006B4A1871519B28DCA480CCA13C7A46477B
:10533000842F133A8544D3477B00470971CDBBF6D0
:10534000D613FFC5BBFE1C34BB8848883605AAA30C
:10535000FFA5B2F013FADCF69CCC2DF4C0998DF2C7
:10536000074E78B58AB8FE10498F2593E079D3218E
:10537000D9F3740AD1F3AAD59E5A44524C88DEB0B0
:105380004CA7F86E9460500FF7277F18BA8C34BB87
:105390003F4B5B625C3C9F0F149131B976C83E5124
:1053A0006557F0C003AFBEA9E5FDC953E83C48907E
:1053B00081ED2151F4EA300E1FA048B5A1ECD6438F
:1053C00069CF5FAC538BB575CC5A83ABD6250D7DB9
:1053D000C04C355D4DCA3078DD2BC4DDE8C4811C7E
:1053E00007AF692B5A71409E8AB09FE763D85E4928
:1053F000F62472EEBAC0030C278E3EE3E220E0D121
:10540000F69DD4141CEB0289AAE263B927979F1F6B
:105410008E540C8B34CFD8F76E90DEB72101E1ADFE
:10542000E8A6FF532FB21A3FA1F6FACCDE8B6A49E9
:10543000D1B0A0A018E7A046A4AE1EA1B2AFE670FE
:10544000748D7700C370EB85BD14BB0DEC3D823BC2
:10545000EF80398AA425BA81DBA30EB16CCAE4B00F
:10546000C4DDFAF5938E3E68719912BF1C60A05C92
:1054700090265509D7370F08BAC85F8D99966C4C9E
:105480008FB237BF61024AE4C6B1AE1E895CE06FDD
:1054900026D229452DDD7B4DE691BF15BC68E2D1B2
:1054A0003FDEB3A1A9A8FD77CEA492E96D4482772F
:1054B00060057E988FFB37198C3CE6D66270794385
:1054C000D092E1D3B74684129712CAEB54352342E7
:1054D000419DDCCAD3084B22F039FF117F3ECB7EC1
:1054E00082FF60166747A910045CD99D0304050A72
:1054F00008060BFF0209070D010C00FF202569209B
:1055000025692025692D256900202025633A256914
:1055100000202020205F5F7C002C004469737020F5
:105520006F66660D0A00555345520046004700421B
:105530004547494E0052414400442E4D59005052B7
:10554000474D00555345522020200066202000671B
:10555000202000424547494E202020202000524173
:105560004420202000442E4D59202020004320209C
:105570002000FFFFFFFF4D0000003B400000000047
:105580000000890F000053400000584000005640C2
:105590000000FF0000003D070000624000006C407A
:1055A00000000A40000000000000F90400007E40F6
:1055B0000000584000008A40000000000000FD0587
:1055C00000008C400000584000009840000000009F
:1055D0000000950700009A40000058400000BB40C2
:1055E000000000000000A5040000BD40000058407D
:1055F00000000F000000F401000002041B0403047B
:1056000001020104020112041A04040400004355BB
:1056100000004B5500004F550000535500002D551C
:1056200000005E550000655500006D5500003E55B8
:10563000000000171B243E42536975180818021910
:105640000219081901180418011A021A0111081187
:105650000212021A081201110411011B021B01108F
:10566000020F0810081B08100410010F0414021484
:105670000115021408150812081504150114041662
:10568000021601170216081708130217041701164D
:1056900004130813040D020C080D0801080D040D75
:1056A000010C040C020C010B020A080B0802020B8D
:1056B000040B010A040A020A010902080809080287
:1056C0000809040901080404020401070807020884
:1056D000020308080107040701030203010602058B
:1056E0000806080408060406010504050205011958
:1056F0000420202020202020202020000000010065
:105700000000265500002B5500002D5500002F5598
:1057100000002D5500003555000039550000B739FF
:0657200000003E550000F0
:00000001FF
